:020000040000FA
:2B000000FFFF62FF2900FFFFFFFFFFFFFFFFFFFFFFFFFFFFFFFFFFFFFFFFFFFFFFFFFFFFFFFFFFFFFFFFFFFFFFFFFF72
:2B002B00C05D96657117D75D96617117D7755D77195C17000000007007D71D96611996657187611986C51DDC6100BC62
:2B005600A0388EE3288EA2380EE1288EA2288AE2108A02000000002884A2100EE1108EE32804E11084A3100A41009929
:2B008100000000000000000000000000000000000000000000000000000000000000000000000000000000000080E7ED
:2B00AC00000000000000000000000000000000000000000000000000000000000000000000000000000000000080E7C2
:2B00D7000020088A0028002008808008080000808000000000000000000000088000088201008000000200000000D780
:2B010200000843201002004006200000000000000000000000000000000000423000018000001000000200000000BD2D
:2B012D00020000000000000000000000000000000000000000000000000000000000000000000000000000000080E540
:2B015800000000000000000000000000000000000000000000000000000000000000000000000000000000000080E715
:2B018300080000000000000000000000000000000000000000000000000000000000000000000000000000000008E75A
:2B01AE00100000000000000000000000000000000000000000000000000000000000000000000000000000000080F79F
:2B01D900040000000000000000000000000000000000000000000000000000000000000000000000000000000080E394
:2B020400000000000000000000000000000000000000000000000000000000000000000000000000000000000080E768
:2B022F00000000000000000000000000000000000000000000000000000000000000000000000000000000000080E73D
:2B025A00000000000000000000000000000000000000000000000000000000000000000000000000000000000080E712
:2B028500000100000000000000000000000000000000000000000000000000000000000000000000000000000090E7D6
:2B02B000180400000000000000000000000000000000000000000000000000000000000000000000000000000090AACD
:2B02DB000010000000000000000000000000000000000000000000000000000000000000000000000000000000A0C484
:2B030600000000000000000000000000000000000000000000000000000000000000000000000000000000000080E765
:2B033100000200000000000000000000000000000000000000000000000000000000000000000000000000000080C55A
:2B035C00000100000000000000000000000000000000000300000000000000000000000000000000000000000080C52D
:2B0387000000421108000000000000800000000000000000010800000000000000000000000000000000000000808A5D
:2B03B200020000000000000000000000000000000000000000000000000000000000000000000000000000000008ED29
:2B03DD00020000000000000000000000000000000000008000040000000000000000000000000000000000000080E906
:2B040800040000000800000000000080000000000000000000000000000000000000000000000000000000000080E3DA
:2B04330002005A170000000000000000000000000000000000002002000000000000000000000000000000000000AD5C
:2B045E00020000000000000000000000000000000000000000000000000000000000000000000000000000000080E50C
:2B048900020000000000000000000000000000000000000000000004000000000000000000000000000000000008AD8D
:2B04B400800008800008800008800008800008800008000000000020000220000220000220000220000220000280E7BA
:2B04DF00800008800008800008800008800008800008000000000020000220000220000220000220000220000280E78F
:2B050A00001000000000000000000000000000000000000000000002000000000000000000000000000000000080C66E
:2B053500620000000000000000000000000000000000000000000002000000000000000000000000000000000080A512
:2B056000820100000000000000000000000000000000000000000000000000000000000000000000000000000088F471
:2B058B00C40101000000000000000000000000000000000000000000000000000000000000000000000000000088A255
:2B05B600820100000000000000000000000000000000000000000000000000000000000000000000000000000088F41B
:2B05E100820100000000000000000000000000000000000000000000000000000000000000000000000000000088F4F0
:2B060C00020000000000000000000000000000000000000000000000000000000000000000000000000000000080E55C
:2B063700000000000000000000000000000000000000000000000000000000000000000000000000000000000080E731
:2B066200801100000000000000000000000000000000000000000000000000000000000000000000000000000000FFDD
:2B068D00E001000000000000000000000000000000000000000040000000000000000000000000000000000000009A87
:2B06B80002000000000000000000000000000000000000000000A000000000000000000000000000000000000008E786
:2B06E300C2210000000000000000000000000000000000000000A000000000000000000000000000000000000088BC25
:2B070E00040200000000000000000000000000000000000000000000000000000000000000000000000000000090D05A
:2B073900020000000000000000000000000000000000000000000000000000000000000000000000000000000008ED9E
:2B076400020000000000000000000000000000000000000000000000000000000000000000000000000000000008ED73
:2B078F00820100000000000000000000000000000000000000000000000000000000000000000000000000000088F440
:2B07BA00000200000000000000000000000000000000000000000000000000000000000000000000000000000080C5CD
:2B07E500600200000000000000000000000000000000000000000000000000000000000000000000000000000080A562
:2B081000000000000000000000000000000000000000000000000000000000000000000000000000000000000080E756
:2B083B00420000000000000000000000000000000000000000000000000000000000000000000000000000000008AD9B
:2B086600820100000000000000000000000000000000000000000000000000000000000000000000000000000088F468
:2B089100840100000000000000000000000000000000000000000000000000000000000000000000000000000010EBBC
:2B08BC00820100000000000000000000000000000000000000000000000000000000000000000000000000000088F412
:2B08E700820100000000000000000000000000000000000000000000000000000000000000000000000000000088F4E7
:2B091200020000000000000000000000000000000000000000000000000000000000000000000000000000000008EDC3
:2B093D00602000000000000000000000000000000000000000000000000000000000000000000000000000000080850A
:2B0968008003000000000000000000000000000000000000000000040000000000000000000000000000000000009C41
:2B099300C003000000000000000000000000000000000000000020000000000000000000000000000000000000009EB8
:2B09BE00020000000000000000000000000000000000000000008000000000000000000000000000000000000008E59F
:2B09E900821100000000000000000000000000000000000000000000000000000000000000000000000000000088F5D3
:2B0A1400040000000000000000000000000000000000000000002000000000000000000000000000000000000090F013
:2B0A3F00820100000000000000000000000000000000000000000000000000000000000000000000000000000088F48D
:2B0A6A00020000000000000000000000000000000000000000000000000000000000000000000000000000000008ED6A
:2B0A9500622000000000000000000000000000000000000000000004000000000000000000000000000000000008CFD9
:2B0AC000800100000000000000000000000000000000000000004000000000000000000000000000000000000000FA50
:2B0AEB00C04100000000000000000000000000000000000000000000000000000000000000000000000000000000BA25
:2B0B1600004000000000000000000000000000000000000000000000000000000000000000000000000000000080E311
:2B0B4100820300000000000000000000000000000000000000000000000000000000000000000000000000000088D6A6
:2B0B6C00020000000000000000000000000000000000000000000000000000000000000000000000000000000008ED67
:2B0B9700840100000000000000000000000000000000000000000000000000000000000000000000000000000010EBB3
:2B0BC200020000000000000000000000000000000000000000000000000000000000000000000000000000000008ED11
:2B0BED0062400000000000000000000000000000000000000000000000000000000000000000000000000000000889AA
:2B0C1800020000000000000000000000000000000000000000000000000000000000000000000000000000000008EDBA
:2B0C4300400000000000000000000000000000000000000000000000000000000000000000000000000000000080A71F
:2B0C6E00800100000000000000000000000000000000000000000000000000000000000000000000000000000000FEDC
:2B0C9900800100000000000000000000000000000000000000000000000000000000000000000000000000000000FEB1
:2B0CC400820100000000000000000000000000000000000000000000000000000000000000000000000000000088F406
:2B0CEF00820100000000000000000000000000000000000000000000000000000000000000000000000000000088F4DB
:2B0D1A00041000000000000000000000000000000000000000000000000000000000000000000000000000000090F317
:2B0D45006201000000000000000000000000000000000000000000000000000000000000000000000000000000089C7C
:2B0D7000820100000000000000000000000000000000000000000000000000000000000000000000000000000088F459
:2B0D9B00420101000000000000000000000000000000000000000000000000000000000000000000000000000008AC35
:2B0DC600800100000000000000000000000000000000000000002000000000000000000000000000000000000000FC65
:2B0DF100002100000000000000000000000000000000000000000000000000000000000000000000000000000080F442
:2B0E1C00002000000000000000000000000000000000000000000000000000000000000000000000000000000080E526
:2B0E4700000300000000000000000000000000000000000000000000000000000000000000000000000000000080D429
:2B0E7200020001000000000000000000000000000000000000000000000000000000000000000000000000000008FD4D
:2B0E9D006200000000000000000000000000000000000000000000000000000000000000000000000000000000088D33
:2B0EC800020000000000000000000000000000000000000000000000000000000000000000000000000000000008ED08
:2B0EF300C22100000000000000000000000000000000000000000000000000000000000000000000000000000088B6B3
:2B0F1E00800100000000000000000000000000000000000000000000000000000000000000000000000000000000FE29
:2B0F4900802300000000000000000000000000000000000000000000000000000000000000000000000000000000DEFC
:2B0F7400000000000000000000000000000000000000000000000000000000000000000000000000000000000080E7EB
:2B0F9F00800100000000000000000000000000000000000000000000000000000000000000000000000000000000FEA8
:2B0FCA00020000000000000000000000000000000000000000000000000000000000000000000000000000000008ED05
:2B0FF500000000000000000000000000000000000000000000000000000000000000000000000000000000000080E76A
:2B102000800008800008800008800008800008800008000000000020000220000220000220000220000220000280E742
:2B104B00800008800008800008800008800008800008000000000020000220000220000220000220000220000280E717
:2B107600000010060000000000000000000000000000000000000000000000000000000000000000000000000080F0C9
:2B10A100000010040000000000000000000000400000000000000000000000000000000000000000000000000080B29E
:2B10CC00004000000000200000000000000000000000802400401200000000000000000000000000000000000000EEB5
:2B10F700000800020000000000000000000000000000000000000000000000000000000000000000000000000000E5DF
:2B112200000810040000200000000000000000400000401200200900000000000000000000000000000000000080C06B
:2B114D00000001000000000000000000000000000000400001000000000000000000000000000000000000000080A70E
:2B117800400001000000000000000000000000000000008000000000000000000000000000000000000000000080BF4C
:2B11A300000000000000000000000000000000000000000000000000000000000000000000000000000000000080E7BA
:2B11CE00000000000000000000000000000000000000000000000000000000000000000000000000000000000080E78F
:2B11F900080400000000000000000000000000000000000000000000000000000000000000000000000000000090BA75
:2B122400000000000000000000000000000000000000000000000000000000000000000000000000000000000090F619
:2B124F00140000000000000000000000000000000000000000000000000000000000000000000000000000000080F3ED
:2B127A00080000000000000000000000000000000000000000000000000000000000000000000000000000000080EFD2
:2B12A500400000000000000000000000000000000000000000000000000000000000000000000000000000000080A7B7
:2B12D000000000000000000000000000000000000000000000000000000000000000000000000000000000000080E78C
:2B12FB000000000000000000000000000000000000000000000000000000000000000000000000000000000000C0A365
:2B132600000000000000000000000000000000000000000000000000000000000000000000000000000000000080E735
:2B135100000000000000000000000000000000000000000000000000000000000000000000000000000000000080E70A
:2B137C00000800000000000000000000000000000000000000000000000000000000000000000000000000000020C559
:2B13A700000000000000000000000000000000000000000000000000000000000000000000000000000000000080E7B4
:2B13D200140000000000000000000000000000000000000000000000000000000000000000000000000000000080F369
:2B13FD00000000000000000000000000000000000000000000000000000000000000000000000000000000000008EFCE
:2B142800000000000000000000000000000000000000000000000000000000000000000000000000000000000080E732
:2B145300000000000000000000000000000000000000000000000000000000000000000000000000000000000080E707
:2B147E00020000000000000000000000000000000000000000000000000000000000000000000000000000000080E5DC
:2B14A900000000000000000000000000000000000000000000000000000000000000000000000000000000000080E7B1
:2B14D400080000000000000000000000000000000000000000000000000000000000000000000000000000000090FE57
:2B14FF00000000000000000000000000000000000000000000000000000000000000000000000000000000000080E75B
:2B152A001E0000000000000000000000000000000000000000000000000000000000000000000000000000000080F9FF
:2B155500000000000000000000000000000000000000000000000000000000000000000000000000000000000080E704
:2B158000000000000000000000000000000000000000000000000000000000000000000000000000000000000080E7D9
:2B15AB00000000000000000000000000000000000000000000000000000000000000000000000000000000000080E7AE
:2B15D600000000000000000000000100000000000000000300000000000000000000000000000000000000000080C5A1
:2B16010000000000000000000008082000004000000080000100000000000000000000000000000000000000008091BC
:2B162C00020000000000000000000000000000000000000000000000000000000000000000000000000000000008ED9C
:2B165700020000000000000000080000000000000000408000000000000000000000000000000000000000000080A579
:2B16820004000000000000000000002000004000000000000000000000000000000000000000000000000000008085D4
:2B16AD00020000000000000000000800000000000000000000002002000000000000000000000000000000000000C71F
:2B16D800020000000000000000000000000000000000000000000000000000000000000000000000000000000080E580
:2B170300020000000000000000000000000000000000000000000004000000000000000000000000000000000008AD00
:2B172E00800008800008800008800008800008800008000000000020000220000220000220000220000220000280E72D
:2B175900800008800008800008800008800008800008000000000020000220000220000220000220000220000280E702
:2B178400000000000000000000000000000000000000000000000002000000000000000000000000000000000080C7F1
:2B17AF00020000000000000000000000000000000000000000000002000000000000000000000000000000000008CD36
:2B17DA00020000000000000000000000000000000000000000000000000000000000000000000000000000000080E57D
:2B180500000000000000000000000000000000000000000000000000000000000000000000000000000000000080E751
:2B183000020000000000000000000000000000000000000000000000000000000000000000000000000000000080E526
:2B185B00020000000000000000000000000000000000000000000000000000000000000000000000000000000080E5FB
:2B188600020000000000000000000000000000000000000000000000000000000000000000000000000000000008ED40
:2B18B100000000000000000000000000000000000000000000000000000000000000000000000000000000000080E7A5
:2B18DC00000000000000000000001000000000000000000000000000000000000000000000000000000000000080E66B
:2B1907000000000000000000006000000000000000000000000040000000000000000000000000000000000000808312
:2B19320002000000000000000000000000000000000000000000A000000000000000000000000000000000000008E7F9
:2B195D0002000000000000000040000000000000000000000000A000000000000000000000000000000000000008A7CE
:2B198800040000000000000000800100000000000000000000000000000000000000000000000000000000000010EBB4
:2B19B300020000000000000000800100000000000000000000000000000000000000000000000000000000000088F40A
:2B19DE00020000000000000000800100000000000000000000000000000000000000000000000000000000000088F4DF
:2B1A0900020000000000000000800100000000000000000000000000000000000000000000000000000000000088F4B3
:2B1A3400000000000000000000000000000000000000000000000000000000000000000000000000000000000080E720
:2B1A5F00000000000000000000000000000000000000000000000000000000000000000000000000000000000080E7F5
:2B1A8A00000000000000000000000000000000000000000000000000000000000000000000000000000000000080E7CA
:2B1AB500020000000000000000000000000000000000000000000000000000000000000000000000000000000008ED0F
:2B1AE000020000000000000000000000000000000000000000000000000000000000000000000000000000000008EDE4
:2B1B0B00040000000000000000000000000000000000000000000000000000000000000000000000000000000090F229
:2B1B3600020000000000000000000000000000000000000000000000000000000000000000000000000000000008ED8D
:2B1B6100020000000000000000000000000000000000000000000000000000000000000000000000000000000008ED62
:2B1B8C00020000000000000000000000000000000000000000000000000000000000000000000000000000000008ED37
:2B1BB700000000000000000000000000000000000000000000000000000000000000000000000000000000000080E79C
:2B1BE200000000000000000000000000000000000000000000000004000000000000000000000000000000000080A7AD
:2B1C0D00000000000000000000000000000000000000000000002000000000000000000000000000000000000080E527
:2B1C3800020000000000000000000000000000000000000000008000000000000000000000000000000000000008E512
:2B1C6300020000000000000000000000000000000000000000000000000000000000000000000000000000000008ED5F
:2B1C8E00040000000000000000000000000000000000000000002000000000000000000000000000000000000090F087
:2B1CB900020000000000000000000000000000000000000000000000000000000000000000000000000000000008ED09
:2B1CE400020000000000000000000000000000000000000000000000000000000000000000000000000000000008EDDE
:2B1D0F00020000000000000000000000000000000000000000000004000000000000000000000000000000000008ADEE
:2B1D3A00000000000000000000000000000000000000000000004000000000000000000000000000000000000080E3DB
:2B1D6500000000000000000000000000000000000000000000000000000000000000000000000000000000000080E7EC
:2B1D9000000000000000000000000000000000000000000000000000000000000000000000000000000000000080E7C1
:2B1DBB00020000000000000000000000000000000000000000000000000000000000000000000000000000000008ED06
:2B1DE600020000000000000000000000000000000000000000000000000000000000000000000000000000000008EDDB
:2B1E1100040000000000000000000000000000000000000000000000000000000000000000000000000000000090F220
:2B1E3C00020000000000000000000000000000000000000000000000000000000000000000000000000000000008ED84
:2B1E6700020000000000000000000000000000000000000000000000000000000000000000000000000000000008ED59
:2B1E9200020000000000000000000000000000000000000000000000000000000000000000000000000000000008ED2E
:2B1EBD00000000000000000000000000000000000000000000000000000000000000000000000000000000000080E793
:2B1EE800000000000000000000000000000000000000000000000000000000000000000000000000000000000080E768
:2B1F1300000000000000000000000000000000000000000000000000000000000000000000000000000000000080E73C
:2B1F3E00020000000000000000000000000000000000000000000000000000000000000000000000000000000008ED81
:2B1F6900000000000000000000000000000000000000000000000000000000000000000000000000000000000008EF56
:2B1F9400000000000000000000000000000000000000000000000000000000000000000000000000000000000090F69C
:2B1FBF00000000000000000000000000000000000000000000000000000000000000000000000000000000000008EF00
:2B1FEA00000000000000000000000000000000000000000000000000000000000000000000000000000000000008EFD5
:2B201500020000000000000000000000000000000000000000000000000000000000000000000000000000000008EDA9
:2B204000000000000000000000000000000000000000000000002000000000000000000000000000000000000080E5F0
:2B206B00000000000000000000000000000000000000000000000000000000000000000000000000000000000080E7E3
:2B209600000000000000000000000000000000000000000000000000000000000000000000000000000000000080E7B8
:2B20C100020000000000000000000000000000000000000000000000000000000000000000000000000000000008EDFD
:2B20EC00000000000000000000000000000000000000000000000000000000000000000000000000000000000080E762
:2B211700000000000000000000000000000000000000000000000000000000000000000000000000000000000080E736
:2B214200000000000000000000000000000000000000000000000000000000000000000000000000000000000080E70B
:2B216D00000000000000000000000000000000000000000000000000000000000000000000000000000000000080E7E0
:2B219800020000000000000000000000000000000000000000000000000000000000000000000000000000000008ED25
:2B21C300000000000000000000000000000000000000000000000000000000000000000000000000000000000080E78A
:2B21EE00000000000000000000000000000000000000000000000000000000000000000000000000000000000080E75F
:2B221900000000000000000000000000000000000000000000000000000000000000000000000000000000000080E733
:2B224400000000000000000000000000000000000000000000000000000000000000000000000000000000000080E708
:2B226F00000000000000000000000000000000000000000000000000000000000000000000000000000000000080E7DD
:2B229A00800008800008800008800008800008800008000000000020000220000220000220000220000220000280E7B6
:2B22C500800008800008800008800008800008800008000000000020000220000220000220000220000220000280E78B
:2B22F000000000000000000000000000000000000000000000000000000000000000000000000000000000000080E75C
:2B231B00000000004000000000000000004000000000000000000000000000000000000000000000000000000080E7B0
:2B234600000000000000000000000000000000000000002400481200000000000000000000000000000000000080CAA4
:2B237100000000004001000000000000004000000000000000000000000000000000000000000000000000000080F749
:2B239C00000000000001000000000000000000000000001200240900000000000000000000000000000000000000E1F5
:2B23C700000000000000000000000000000000000000400001000000000000000000000000000000000000000080B773
:2B23F200000000000000000000000000000000000000008000000000000000000000000000000000000000000080EFD1
:2B241D00000000000000000000000000000000000000000000000000000000000000000000000000000000000080E72D
:2B244800000000000000000000000000000000000000000000000000000000000000000000000000000000000080E702
:2B2473000000000000000000000000000000000000000000000000000000000000000000000000000000000000E081DD
:2B249E000000000000000000000000000000000000000000000000000000000000000000000000000000000000C0A3B0
:2B24C900000000000000000000000000000000000000000000000000000000000000000000000000000000000080E781
:2B24F4000000000000000000000000000000000000000000000000000000000000000000000000000000000000A0C558
:2B251F00000000000000000000000000000000000000000000000000000000000000000000000000000000000080E72A
:2B254A00000000000000000000000000000000000000000000000000000000000000000000000000000000000090F6E0
:2B257500100000000000000000000000000000000000000000000000000000000000000000000000000000000080F7B4
:2B25A000000000000000000000000000000000000000000000000000000000000000000000000000000000000080E7A9
:2B25CB00000000000000000000000000000000000000000000000000000000000000000000000000000000000080E77E
:2B25F600080000000000000000000000000000000000000000000000000000000000000000000000000000000080EF43
:2B262100000000000000000000000000000000000000000000000000000000000000000000000000000000000080E727
:2B264C00140000000000000000000000000000000000000000000000000000000000000000000000000000000080F3DC
:2B267700000000000000000008000000090000000000000000000000000000000000000000000000000000000000E641
:2B26A200020000000000000000000000000000000400000000000000000000000000000000000000000000000080A1E6
:2B26CD00080000000000000000000000000000000000000000000000000000000000000000000000000000000080EF6B
:2B26F800000000000000000000000000000000000000000000000000000000000000000000000000000000000008EFC0
:2B272300000000000000000000000000000000000000000000000000000000000000000000000000000000000080E724
:2B274E00000000000000000000000000000000000000000000000000000000000000000000000000000000000080E7F9
:2B277900000000000000000000020000000000000000000000000000000000000000000000000000000400000080A10E
:2B27A4001C0000000000000010000040000000008000000000000000000000000000000000000000000000000080A6F8
:2B27CF00000000000000000000000000000000000000000000000000000000000000000000000000000000000080E778
:2B27FA00000000000000000000000000000000000000000000000000000000000000000000000000000400000080A38D
:2B282500000000000000000024000020000000000C00000000000000000000000000000000000000000800000080E3CD
:2B285000000000000000000000000000000000000000000000000000000000000000000000000000000000000080E7F6
:2B287B002000000000002800180088E4000882000096080000000000002000000000000000000000000000000080831B
:2B28A6002200000000002020000000000000020000040000000000000000000000000000000000000000000000088F08
:2B28D100020000000000080000040000000000000000000000000000000000000000000000000000000000000080E965
:2B28FC00040000000000000010008800000880000010000000000000002000000000000000000000000000000000E974
:2B2927000200000000000020000000E400000000009A0E0000000000000000000000000000000000000000000000F6E1
:2B295200020000000000000000000000000000000000000000000000000000000000000000000000000000000080E5F3
:2B297D00020000000000000000000000000000000000000000000000000000000000000000000000000000000008ED38
:2B29A800800008800008800008800008800008800008000000000020000220000220000220000220000220000280E7A1
:2B29D300800008800008800008800008800008800008000000000020000220000220000220000220000220000280E776
:2B29FE00000000000000000000000000000000000000000000000000000000000000000000000000000000000080E747
:2B2A2900020000000000000046000000000000608000000000000000000000000000000000000000000000000080A931
:2B2A5400020000000000000000000000000000800300000000000000000000000000000000000000000000000088D674
:2B2A7F0004000000000000001C020000000000C00300000000000000000000000000000000000000000000000008CB74
:2B2AAA00020000000000000018010000000000800100000000000000000000000000000000000000000000000008EC71
:2B2AD500020000000000000018000000000000800100000000000000000000000000000000000000000000000008ED46
:2B2B0000020000000000000000000000000000000000000000000000000000000000000000000000000000000080E543
:2B2B2B00000000000000000018000000000000000000000000000000000000000000000000000000000000000000FE69
:2B2B5600000000000000000000000000000000000000000000000000000000000000000000000000000000000080E7ED
:2B2B810000000000000000001E0800060400006081000000000000000000000000000000000000000000000000008B8D
:2B2BAC00020000000000000000040020000000800300000000000000000000000000000000000000000000000000F85D
:2B2BD70002000000000000001C000024000000400300000000000000000000000000000000000000000000000088A521
:2B2C0200040000000000000000000000040000800100000000000000000000000000000000000000000000000088F6A0
:2B2C2D00020000000000000018010020000000002300000000000000000000000000000000000000000000000088E6B0
:2B2C5800020000000000000018000000000000008000000000000000000000000000000000000000000000000088FC33
:2B2C8300020000000000000000000010100000000300000000000000000000000000000000000000000000000080D7AA
:2B2CAE00000000000000000000000000000000000000000000000000000000000000000000000000000000000080E794
:2B2CD90000000000000000002601001E040000600400000000000000000000000000000000000000000000000000FD26
:2B2D0400000000000000000000000020000000000000000000000000000000000000000000000000000000000080C53F
:2B2D2F0002000000000000001C02003C000000C02300000000000000000000000000000000000000000000000088B4FE
:2B2D5A00020000000000000038000000040000802100000000000000000000000000000000000000000000000008C99E
:2B2D8500040000000000000018000038000000800300000000000000000000000000000000000000000000000010EB51
:2B2DB000020000000000000000000018000000000000000000000000000000000000000000000000000000000088F462
:2B2DDB00020000000000000018000000000000800100000000000000000000000000000000000000000000000008ED3D
:2B2E0600020000000000000000000000100000000000000000000000000000000000000000000000000000000008FD8A
:2B2E31000000000000000000A6000006000000600001000000000000000000000000000000000000000000000000B5B4
:2B2E5C00000000000000000000000000000000000000000000000000000000000000000000000000000000000080E7E4
:2B2E870000000000000000001C02001C020000C023000000000000000000000000000000000000000000000000009E63
:2B2EB200020000000000000018080018000000800100000000000000000000000000000000000000000000000000F446
:2B2EDD00020000000000000038000038100000802100000000000000000000000000000000000000000000000088E639
:2B2F0800040000000000000000000000000000000000000000000000000000000000000000000000000000000008EBA7
:2B2F3300020000000000000018000018000000800100000000000000000000000000000000000000000000000088F444
:2B2F5E00020000000000000000000000000000001000000000000000000000000000000000000000000000000008EC42
:2B2F8900020000000000000006080006040000600200000000000000000000000000000000000000000000000080AB76
:2B2FB400000000000000000018040038000000000000000000000000000000000000000000000000000000000080C15D
:2B2FDF0000000000000000001C00003C000000C02300000000000000000000000000000000000000000000000000BCD0
:2B300A00000000000000000018000018000000800100000000000000000000000000000000000000000000000000FEEC
:2B303500000000000000000018000018000000801100000000000000000000000000000000000000000000000000FFB0
:2B306000020000000000000000000000000000000000000000000000000000000000000000000000000000000008ED4E
:2B308B00020000000000000000000000000000800100000000000000000000000000000000000000000000000088F41B
:2B30B600020000000000000010000000000000000000000000000000000000000000000000000000000000000008FCD9
:2B30E100020000000000000016080016040000E081000000000000000000000000000000000000000000000000889011
:2B310C00000000000000000010040038000000000200000000000000000000000000000000000000000000000000EB5F
:2B313700000000000000000014000034000000C00300000000000000000000000000000000000000000000000000BEA4
:2B316200000000000000000010000018000000000001000000000000000000000000000000000000000000000000FF1A
:2B318D00000000000000000010010010020000800300000000000000000000000000000000000000000000000000DF92
:2B31B800020000000000000010080000020000800100000000000000000000000000000000000000000000000088EFD8
:2B31E300000000000000000008000030000000000000000000000000000000000000000000000000000000000088D42D
:2B320E00000000000000000000000010000000000000000000000000000000000000000000000000000000000090E70E
:2B3239000000000000000000060800160400006080000000000000000000000000000000000000000000000000089AC0
:2B326400000000000000000000040030000000000200000000000000000000000000000000000000000000000008FA07
:2B328F00020000000000000004000034000000400200000000000000000000000000000000000000000000000008BCD4
:2B32BA00000000000000000000000010040000000001000000000000000000000000000000000000000000000080E272
:2B32E500000000000000000000010030000000000200000000000000000000000000000000000000000000000080F714
:2B331000000000000000000000080010000000000000000000000000000000000000000000000000000000000080FEFC
:2B333B00000000000000000010000008100000004300000000000000000000000000000000000000000000000000D923
:2B336600020000000000000000000000010000000100000000000000000000000000000000000000004000000008F9F7
:2B339100020000000000000016080006000000608100000000000000000000000000000000000000800100000088946D
:2B33BC00020000000000000018040000000000000300000000000000000000000000000000000000000000000088C37A
:2B33E70002000000000000001400001C020000400300000000000000000000000000000000000000008700000088EB4A
:2B3412000000000000000000180000180000000001010000000000000000000000000000000000000006000000808057
:2B343D00000000000000000010020018080000000300000000000000000000000000000000000000004600000000B435
:2B346800000000000000000000000000000000000100000000000000000000000000000000000000000000000080F6C2
:2B3493000000000000000000301000180000008042000000000000000000000000000000000000000006000000B0A698
:2B34BE000A000000000000000000000000000000000000000000000000000000000000000000000000000000006883EE
:2B34E900000000000000000000000000000000000000000000000000000000000000000000000000000000000080E751
:2B351400800008800008800008800008800008800008000000000020000220000220000220000220000220000280E729
:2B353F00800008800008800008800008800008800008000000000020000220000220000220000220000220000280E7FE
:2B356A000000000000000020200860400000000000000400000000000000000000000000000000000000000000808941
:2B359500000000000000000000000000000000004100040000000000000000000000000100000000000000000080E75E
:2B35C000000002000020000000004020000002200000000000000000000000000000000000000000000000000080C3F9
:2B35EB000000000010000000000020000008008000000000000000000000004000000000000000000002000000808EAD
:2B361600000002001020002028080068000802204100040000000000000000400000000100000000000000000000EA05
:2B364100000000000000000000000000000000000300000000000000000000000000000000000000000000000080D407
:2B366C00000000000000000000000010000000400000000000000000000000000000000000000000000000000080B6AD
:2B369700000000000000000000000000000000000000000000000000000000000000000000000000000000000080E7A1
:2B36C200000000000000000000010000100000004000000000000000000000000000000000000000000000000080F21A
:2B36ED00100000000000000000080000000000000000000000000000000000000000000000000000000000000080FF1B
:2B371800000000000000000000020004000000000000000000000000000000000000000000000000000000000080A55B
:2B374300000000000000000000000000020000000000000000000000000000000000000000000000000000000080E5F4
:2B376E00000000000000000000000000000000800000000000000000000000000000000000000000000000000000EFC1
:2B379900000000000000000010000000100000000000000000000000000000000000000000000000000000000080E67F
:2B37C400100000000000000000000000000000000000000000000000000000000000000000000000000000000090E654
:2B37EF00000000000000000000000000000000002001000000000000000000000000000000000000000000000080F519
:2B381A00000000000000000000040000000000000000000000000000000000000000000000000000000000000080E31C
:2B384500000000000000000000000000000000000000000000000000000000000000000000000000000000000080E7F1
:2B387000000000000000000000000080000000000000000000000000000000000000000000000000000000000000E7C6
:2B389B000000000000000000000000000000000000000000000000000000000000000000000000000000000000A0C59D
:2B38C600000000000000000000000000000000000000000000000000000000000000000000000000000000000090F651
:2B38F100000000000000000000000000000000000000000000000000000000000000000000000000000000000080E745
:2B391C00000000000000000000000000000000000000000000000000000000000000000000200000000000000080C719
:2B394700080000000000000000000000000000000000000000000000000000000000000000010000000000000080EEDE
:2B397200120000000000000000000000000000000000000000000000000000000000000000000000000000000008FD13
:2B399D00000000000000000000000000000000000000000000000000000000000000000000000000000000000080E798
:2B39C800000000000000000000000000000000000000000000000000000000000000000000000000000000000080E76D
:2B39F300040000000000000000000000000000000000000000000000000000000000000000000000000000000080E342
:2B3A1E001400000000000000000000000000000000000000000000000000000000000000400000000000000000388C65
:2B3A4900000000000000000000000000000000000000000000000000000000000000000000000000000000000080E7EB
:2B3A7400000000000000000000000000000000000000000000000000000000000000000000000000000000000080E7C0
:2B3A9F00000000000000000000000000000000000000000000000000000000000000000080000000000000000000E795
:2B3ACA00000000000000000000000000000000000000000300000000000000000000000000000000000000000080D47A
:2B3AF500000000000000000000000000000000000000800000481008800000000000000010004900000000000080A2CB
:2B3B2000020000000000000000000000000000000000000000000008800000000000000010080000000000000008F4DC
:2B3B4B000200000000000000000000000000000000004000002408000000000000000000000000000000000000008160
:2B3B7600040000000000000000000000000000000000000000000000000000000000000000000000000000000080E3BD
:2B3BA10002000000000000000000000000000000000000000000200200000000000000000000CF00000000000000BC4A
:2B3BCC00020000000000000000000000000000000000000000000000000000000000000000000000000000000080E567
:2B3BF700020000000000000000000000000000000000000000000004000000000000000000000000000000000008ADE8
:2B3C2200800008800008800008800008800008800008000000000020000220000220000220000220000220000280E714
:2B3C4D00800008800008800008800008800008800008000000000020000220000220000220000220000220000280E7E9
:2B3C7800000000000000000000000000000000000000000000000002000000000000000000000000000000000080C7D8
:2B3CA300020000000000000000000000000000000000000000000002000000000000000018400000000000000088947E
:2B3CCE00020000000000000000000000000000000000000000000000000000000000000000000000000000000008EDD4
:2B3CF9000400000000000000000000000000000000000000000000000000000000000000700800000000000000908D07
:2B3D24000200000000000000000000000000000000000000000000000000000000000000601000000000000000089B5F
:2B3D4F000200000000000000000000000000000000000000000000000000000000000000E00000000000000000888B54
:2B3D7A00020000000000000000000000000000000000000000000000000000000000000000000000000000000008ED27
:2B3DA5000000000000000000000000000000000000000000000000000000000000000000600000000000000000808192
:2B3DD000000000000000000000000000000000000000000000000000000000000000000000200000000000000080C761
:2B3DFB00000000000000000000000000000000000000000000004000000000000000000098000000000000000080FA4B
:2B3E260002000000000000000000000000000000000000000000A000000000000000000000000000000000000008E7E0
:2B3E510002000000000000000000000000000000000000000000A000000000000000000090200000000000000088D696
:2B3E7C00040000000000000000000000000000000000000000000000000000000000000080000000000000000010F295
:2B3EA700020000000000000000000000000000000000000000000000000000000000000080000000000000000088EDF9
:2B3ED200020000000000000000000000000000000000000000000000000000000000000000400000000000000008ADCE
:2B3EFD000200000000000000000000000000000000000000000000000000000000000000C0000000000000000088A9A7
:2B3F2800000000000000000000000000000000000000000000000000000000000000000000200000000000000080C707
:2B3F5300000000000000000000000000000000000000000000000000000000000000000098000000000000000080FE2D
:2B3F7E0000000000000000000000000000000000000000000000000000000000000000006000000000000000008081B7
:2B3FA9000200000000000000000000000000000000000000000000000000000000000000F0200000000000000088BA99
:2B3FD4000200000000000000000000000000000000000000000000000000000000000000600000000000000000088BCD
:2B3FFF00040000000000000000000000000000000000000000000000000000000000000060000000000000000090940F
:2B402A00020000000000000000000000000000000000000000000000000000000000000000000000000000000008ED74
:2B405500020000000000000000000000000000000000000000000000000000000000000000000000000000000008ED49
:2B408000020000000000000000000000000000000000000000000000000000000000000000200000000000000008CD1E
:2B40AB000000000000000000000000000000000000000000000000000000000000000000F800000000000000008098DA
:2B40D600000000000000000000000000000000000000000000000004000000000000000000000000000000000080A794
:2B4101000000000000000000000000000000000000000000000020000000000000000000F0200000000000000000B2B1
:2B412C00020000000000000000000000000000000000000000008000000000000000000080000000000000000088E5F9
:2B4157000200000000000000000000000000000000000000000000000000000000000000E00000000000000000888B48
:2B4182000400000000000000000000000000000000000000000020000000000000000000600000000000000000909668
:2B41AD00020000000000000000000000000000000000000000000000000000000000000000000000000000000008EDF0
:2B41D800020000000000000000000000000000000000000000000000000000000000000000000000000000000008EDC5
:2B420300020000000000000000000000000000000000000000000004000000000000000018020000000000000088B632
:2B422E00000000000000000000000000000000000000000000004000000000000000000000000000000000000080E3C2
:2B42590000000000000000000000000000000000000000000000000000000000000000007008000000000000008098AA
:2B42840000000000000000000000000000000000000000000000000000000000000000006000000000000000008081AE
:2B42AF000200000000000000000000000000000000000000000000000000000000000000E008000000000000008883EF
:2B42DA00020000000000000000000000000000000000000000000000000000000000000000000000000000000008EDC2
:2B4305000400000000000000000000000000000000000000000000000000000000000000600000000000000000909405
:2B433000020000000000000000000000000000000000000000000000000000000000000000200000000000000008CD6B
:2B435B000200000000000000000000000000000000000000000000000000000000000000D8000000000000000008B0A5
:2B4386000200000000000000000000000000000000000000000000000000000000000000600000000000000000088B17
:2B43B1000000000000000000000000000000000000000000000000000000000000000000D0200000000000000000925F
:2B43DC000000000000000000000000000000000000000000000000000000000000000000600000000000000000808155
:2B440700000000000000000000000000000000000000000000000000000000000000000040080000000000000080AB17
:2B443200020000000000000000000000000000000000000000000000000000000000000080000000000000000088ED68
:2B445D00000000000000000000000000000000000000000000000000000000000000000040000000000000000008AB41
:2B4488000000000000000000000000000000000000000000000000000000000000000000402000000000000000909287
:2B44B3000000000000000000000000000000000000000000000000000000000000000000D8000000000000000008B24C
:2B44DE00000000000000000000000000000000000000000000000000000000000000000040000000000000000008ABC0
:2B4509000200000000000000000000000000000000000000000000000000000000000000D02000000000000000889875
:2B4534000000000000000000000000000000000000000000000020000000000000000000C0000000000000000000A1DB
:2B455F000000000000000000000000000000000000000000000000000000000000000000C0000000000000000000A3CE
:2B458A00000000000000000000000000000000000000000000000000000000000000000040400000000000000080E323
:2B45B5000000000000000000000000000000000000000000000000000000000000000000A0000000000000000000C576
:2B45E000020000000000000000000000000000000000000000000000000000000000000000010000000000000008ECB9
:2B460B00020000000000000000000000000000000000000000000000000000000000000098000000000000000008F4EE
:2B463600020000000000000000000000000000000000000000000000000000000000000000000000000000000008ED62
:2B466100020000000000000000000000000000000000000000000000000000000000000070080000000000000008921A
:2B468C00000000000000000000000000000000000000000000000000000000000000000060040000000000000080859A
:2B46B7000000000000000000000000000000000000000000000000000000000000000000600000000000000000808177
:2B46E200000000000000000000000000000000000000000000000000000000000000000000000000000000000080E746
:2B470D000000000000000000000000000000000000000000000000000000000000000000600000000000000000808120
:2B473800020000000000000000000000000000000000000000000000000000000000000000000000000000000008ED5F
:2B476300000000000000000000000000000000000000000000000000000000000000000000000000000000000080E7C4
:2B478E00800008800008800008800008800008800008000000000020000220000220000220000220000220000280E79D
:2B47B900800008800008800008800008800008800008000000000020000220000220000220000220000220000280E772
:2B47E4000000000000000000000000000000000000000000000000000000000000000000002084010000000000809BEA
:2B480F00000000000000000000000000100000000400000000000000000000000000000000000400000000000080F7EF
:2B483A000000000000000000000000000000000000000024010002000000000000080000080000010000000000808318
:2B486500000000000000000000000000000000000000000000000000000000000000000000008000000000000080EF39
:2B489000000000000000000000000000100000000400009200000100000000000008000008200400000000000080EDB5
:2B48BB00000000000000000000000000000000000000400001000000000000000000000000000000000000000080B75A
:2B48E600000000000000000000000000000000000000008000000000000000000000000010000000000000000080FE99
:2B491100000000000000000000000000000000000000000000000000000000000000000000000000000000000080E714
:2B493C00000000000000000000000000000000000000000000000000000000000000000000000000000000000080E7E9
:2B496700000000000000000000000000000000000000000000000000000000000000000000100000000000000080F79E
:2B499200000000000000000000000000000000000000000000000000000000000000000000000000000000000080E793
:2B49BD00000000000000000000000000000000000000000000000000000000000000000000400000000000000090B649
:2B49E800000000000000000000000000000000000000000000000000000000000000000000100000000000000080F71D
:2B4A13000000000000000000000000000000000000000000000000000000000000000000100000000000000000C0B2F6
:2B4A3E00000000000000000000000000000000000000000000000000000000000000000000000000000000000080E7E6
:2B4A6900100000000000000000000000000000000000000000000000000000000000000000000000000000000080F79B
:2B4A9400000000000000000000000000000000000000000000000000000000000000000000000000000000000080E790
:2B4ABF000000000000000000000000000000000000000000000000000000000000000000000000000000000000A0C567
:2B4AEA00080000000000000000000000000000000000000000000000000000000000000000020000000000000080ED2A
:2B4B1500000000000000000000000000000000000000000000000000000000000000000000000000000000000090F6EF
:2B4B4000000000000000000000000000000000000000000000000000000000000000000000000000000000000008EF53
:2B4B6B00000000000000000000000000000000000000000000000000000000000000000000000000000000000080E7B8
:2B4B9600080000000000000000000800000000000000000000000000000000001000000000000000000000000000EEE6
:2B4BC100000000000000000000000000000000000000000000000000000000000000000000000000000000000080E762
:2B4BEC00000000000000000000000000000000000000000000000000000000000000000000000000000000000080E737
:2B4C1700000000000000000000000000000000000000000000000000000000000000000000000000000000000080E70B
:2B4C4200000000000000000000000000000000000000000000000000000000000000000000000000000000000080E7E0
:2B4C6D00000000000000000000000000000000000000000000000000000000000000000000000000000000000080E7B5
:2B4C9800000000000000000000000000000000000000000000000000000000000200000000000000000000000008CD1A
:2B4CC300000000000000000000000000000000000000000000000000000000000000000000000000000000000080E75F
:2B4CEE00000000000000000000000000000000000000000000000000000000000000000000000000000000000080E734
:2B4D1900000000000000000000000200000000000000000000000000000000002800000000000000000000000000C77E
:2B4D4400000000000000000000000000000000000000000000000000000000000000000000000000000000000080E7DD
:2B4D6F00000000000000000000000080200000000000000000000000000000800800000000020000002000020000CD00
:2B4D9A00000000000000000000000000200000000000000000000000000000008000000000000000000000000008C77F
:2B4DC500020000000000000000004010000000000000000000000000000000100000000000020000000000000080E2FD
:2B4DF000020000000000000000000000000000000000000000000000000000000000000000000000002000020080E50F
:2B4E1B00020000000000000000000090020000000000000000000000000000900800000000000000000000000000EE52
:2B4E4600020000000000000000000000000000000000000000000000000000000000000000000000000000000080E5DA
:2B4E7100000000000000000000000000000000000000000000000000000000000000000000000000000000000008EF1F
:2B4E9C00800008800008800008800008800008800008000000000020000220000220000220000220000220000280E788
:2B4EC700800008800008800008800008800008800008000000000020000220000220000220000220000220000280E75D
:2B4EF200000000000000000000000000000000000000000000000000000000000000000000000000000000000080E72E
:2B4F1D00020000000000000000E00B00000000000000000000000000000000800F01000000000000000000000080D19B
:2B4F4800020000000000000000001000000000000000000000000000000000000400000000000000000000000008A878
:2B4F7300040000000000000000C00100000000000000000000000000000000008500000000000000000000000088EF52
:2B4F9E00020000000000000000000200000000000000000000000000000000004600000000000000000000000008ADE9
:2B4FC900020000000000000000800100000000000000000000000000000000000800000000000000000000000008F436
:2B4FF400020000000000000000800100000000000000000000000000000000008400000000000000000000000000B0DB
:2B501F00000000000000000000000000000000000000000000000000000000000C00000000000000000000000000A3B7
:2B504A00000000000000000000000000000000000000000000000000000000000800000000000000000000000000E74C
:2B5075000000000000000000006080000000000000000000000000000000008001000000000000000000000000009619
:2B50A000000000000000000000000001000000000000000000000000000000000000000000000000000000000008FFDD
:2B50CB00020000000000000000400000000000000000000000000000000000008700000000000000000000000008D217
:2B50F600020000000000000000000000000000000000000000000000000000000604000000000000000000000090D221
:2B512100020000000000000000001200000000000000000000000000000000000E00000000000000000000000088A811
:2B514C00020000000000000000004000000000000000000000000000000000000000000000000000000000000008E905
:2B517700000000000000000000000300000000000000000000000000000000000600000000000000000000000008BA42
:2B51A200000000000000000000000000000000000000000000000000000000001000000000000000000000000080E66C
:2B51CD00000000000000000000E00B00000000000000000000000000000000800900000000000000000000000080A51E
:2B51F800000000000000000000000100000000000000000000000000000000000000000000000000000000000080F615
:2B522300000000000000000000402100000000000000000000000000000000008700000000000000000000000008C3AD
:2B524E000200000000000000008011000000000000000000000000000000000006000000000000000000000000889381
:2B527900020000000000000000000000000000000000000000000000000000004600000000000000000000000090969C
:2B52A400020000000000000000000100000000000000000000000000000000000000000000000000000000000008FCD8
:2B52CF00020000000000000000008300000000000000000000000000000000000600000000000000000000000008B071
:2B52FA00000000000000000000000100000000000000000000000000000000000000000000000000000000000008FE82
:2B532500000000000000000000600B00000000000000000000000000000000801700000000000000000000000080CA11
:2B535000000000000000000000001100000000000000000000000000000000000400000000000000000000000080B3EA
:2B537B00000000000000000000400100000000000000000000000000000000008500000000000000000000000080EBD6
:2B53A600020000000000000000000300000000000000000000000000000000000604000000000000000000000080F05D
:2B53D100020000000000000000000100000000000000000000000000000000000000000000000000000000000008FCAA
:2B53FC00040000000000000000001100000000000000000000000000000000000401000000000000000000000008AFB5
:2B542700020000000000000000800200000000000000000000000000000000000C00000000000000000000000008833F
:2B545200020000000000000000000000000000000000000000000000000000000000000000000000000000000008ED38
:2B547D00020000000000000000600A00000000000000000000000000000000800F01000000000000000000000000C840
:2B54A800000000000000000000801100000000000000000000000000000000004000000000000000000000000000FB0D
:2B54D300000000000000000000C00100000000000000000000000000000000000F00000000000000000000000080C995
:2B54FE00000000000000000000800100000000000000000000000000000000000800000000000000000000000080FE7C
:2B552900000000000000000000800100000000000000000000000000000000000E000000000000000000000000089030
:2B5554000200000000000000000000000000000000000000000000000000000006000000000000000000000000088B91
:2B557F00020000000000000000000000000000000000000000000000000000000000000000000000000000000090F47B
:2B55AA00020000000000000000000000000000000000000000000000000000000000000000000000000000000008EDDF
:2B55D500020000000000000000E0810000000000000000000000000000000080090100000000000000000000008895A1
:2B560000000000000000000000000001000000000000000000000000000000004000000000000000000000000008FB3B
:2B562B00000000000000000000C00100000000000000000000000000000000000900000000000000000000000080AF5B
:2B565600000000000000000000000000000000000000000000000000000000000800000000000000000000000000E73A
:2B568100000000000000000000801300000000000000000000000000000000000800000000000000000000000080DD06
:2B56AC00000000000000000000800100000000000000000000000000000000000002000000000000000000000000DE72
:2B56D700020000000000000000000000000000000000000000000000000000000C00000000000000000000000088A969
:2B570200020000000000000000000100000000000000000000000000000000000400000000000000000000000008B8B5
:2B572D00020000000000000000608100000000000000000000000000000000800D01000000000000000000000008D9FF
:2B575800020000000000000000000101000000000000000000000000000000004400000000000000000000000008AC2A
:2B578300000000000000000000400100000000000000000000000000000000000D00000000000000000000000000E3CA
:2B57AE00000000000000000000000100000000000000000000000000000000000C00000000000000000000000000B211
:2B57D900000000000000000000001300000000000000000000000000000000000C0000000000000000000000000091F5
:2B580400000000000000000000004100000000000000000000000000000000000402000000000000000000000080961C
:2B582F00020000000000000000800200000000000000000000000000000000000A00000000000000000000000008E5D3
:2B585A00020000000000000000000000000000000000000000000000000000000000000000000000000000000008ED2C
:2B5885000400000000000000006080000000000000000000000000000000008009010000000000000000000000909367
:2B58B00002000000000000000080010100000000000000000000000000000000460000000000000000000000008886F5
:2B58DB00020000000000000000C00100000000000000000000000000000000000F00000000000000000000000008C305
:2B59060002000000000000000080010000000000000000000000000000000000060000000000000000000000008892D3
:2B593100000000000000000000800100000000000000000000000000000000000600000000000000000000000000982C
:2B595C00000000000000000000000000000000000000000000000000000000000000000000000000000000000080E7B9
:2B5987001600000000000000000000000000000000000000000000000000000000000000000000000000000000A0D36C
:2B59B2000C00000000000000000000000000000000000000000000000000000000000000000000000000000000D0BE30
:2B59DD00000000000000000000000000000000000000000000000000000000000000000000000000000000000080E738
:2B5A0800800008800008800008800008800008800008000000000020000220000220000220000220000220000280E710
:2B5A3300800008800008800008800008800008800008000000000020000220000220000220000220000220000280E7E5
:2B5A5E00000000000000000000208000070000000000000000000000000000904000000000000000000000000000D4D2
:2B5A8900000000000000000000000000000000000000000000000000000000100400000000000000000000000080B3AB
:2B5AB400000000000000000000000000040000000000000000000000000000000000000000000000000100000080F250
:2B5ADF00000000000000000000000000000000000000000000000000004000000000000000000000020000000080E1F9
:2B5B0A000000000000000000002080000100000000000000000000000040009044000000000000000201000000008137
:2B5B3500000000000000000000000000000000000000000000000000000000000400000000000000000000000080A31E
:2B5B6000000000000000000000800001000000000000000000000000000000000004000000000000000000000000BFD6
:2B5B8B00000000000000000000C04000000000000000000000000000000000000000000000000000000000000000AB44
:2B5BB600000000000000000000000000000000000000000000000000000000000003000000000000000000000080D76A
:2B5BE100020000000000000000000000000000000000000000000000000000000000000000000000000000000080E532
:2B5C0C00000000000000000000000000000000000000000000000000000000000100000000000000000000000080F6F6
:2B5C3700000000000000000000000000000000000000000000000000000000000000000000000000000000000080E7DB
:2B5C6200000000000000000000000000000000000000000000000000000000000000000000000000000000000080E7B0
:2B5C8D00100000000000000000000000000000000000000000000000000000000100000000000000000000000008EEE5
:2B5CB8000200000000000000000000000000000000000000000000000000000000000000000000000000000000A0C758
:2B5CE300000000000000000000000000000000000000000000000000000000000000000000000000000000000080E72F
:2B5D0E00000000000000000000000000000000000000000000000000000000000000000000000000000000000080E703
:2B5D3900000000000000000000002000000000000000000000000000000000000000000000000000000000000080E5BA
:2B5D6400000000000000000000000100000000000000000000000000000000002000000000000000000000000080F47F
:2B5D8F000C0000000000010000000000000000000000000000000000000000000000000000000000000000000080EA72
:2B5DBA00020000000000000000000000000000000000000000000000000000000000000000000000000000000080E557
:2B5DE5001000000000000000000000000000000000000000000000000000000000000000000000000000000000A0D50E
:2B5E10000000000000600000000000000000000000000000000000000000000000000000000000000000000000088976
:2B5E3B00000000000000040000000000000000000000000000000000000000000000000000000000000000000080E3D5
:2B5E6600000000000000000000000000000000000000000000000000000000000000000000000000000000000080E7AA
:2B5E9100000000000000000000000000000000000000000000000000000000000000000000000000000000000080E77F
:2B5EBC00000000000000000000000000000000000000000000000000000000000000000000000000000000000080E754
:2B5EE700000000000000000000000000000000000000000000000000000000000000000000000000000000000090F60A
:2B5F12001A0000000000000000000000000000000000000000000000000000000000000000000000000000000090ECCE
:2B5F3D00000000000000000000000000000000000000000000000000000000000000000000000000000000000080E7D2
:2B5F6800000000000000000000000000000000000000000000000000000000000000000000000000000000000080E7A7
:2B5F9300000000000020000000000000000000000000000000000000000000000000000800000000000000000000C5F6
:2B5FBE00000000000000000000000000000000000000000300000000000000000000000C000000000000000000009019
:2B5FE9000000000020A2000000000020000000000000012000081200000000000000808004000000000000000080AD3F
:2B601400020000000000000000000000000010000000000000000000000000000000000000000000000000000008FC4B
:2B603F00020000000000040000000000000000000000001000040900000000000000000000000000000000000000F51E
:2B606A00040000000080000000000020000010000000010000000000000000000000000000000000000000000000D185
:2B6095000200000020220000000000000000000000000000000020020000000000008000040000000000000000008F67
:2B60C000020000000000000000000000000000000000000000000000000000000000000000000000000000000080E54E
:2B60EB00020000000000000000000000000000000000000000000004000000000000000000000000000000000008ADCF
:2B611600800008800008800008800008800008800008000000000020000220000220000220000220000220000280E7FB
:2B614100800008800008800008800008800008800008000000000020000220000220000220000220000220000280E7D0
:2B616C0000000000000010000000000000000000000000000000000200000000000000240000000000000000008091C1
:2B619700020000000006000000000000000000000000000000000002000000000000800500000000000000000088F0D6
:2B61C200020000000000000000000000000000000000000000000000000000000000008400000000000000000008A183
:2B61ED00040000000004010000000000000000000000000000000000000000000000000500000000000000000090E603
:2B621800020000000000040000000000000000000000000000000000000000000000000404000000000000000008ED58
:2B624300020000000000000000000000000000000000000000000000000000000000000C00000000000000000088A9F1
:2B626E00020000000000020000000000000000000000000000000000000000000000000400000000000000000008AB4A
:2B629900000000000030000000000000000000000000000000000000000000000000000A04000000000000000000B6E6
:2B62C400000000000000020000000000000000000000000000000000000000000000004000000000000000000080E10C
:2B62EF00000000000006000000000000000000000000000000004000000000000000800700000000000000000000FCBB
:2B631A0002000000000000000000000000000000000000000000A000000000000000000000000000000000000008E7C7
:2B63450002000000001C02000000000000000000000000000000A0000000000000000007040000000000000000888B4F
:2B637000040000000018000000000000000000000000000000000000000000000000000800000000000000000090EB63
:2B639B00020000000038080000000000000000000000000000000000000000000000000600000000000000000088B84F
:2B63C6000200000000000000000000000000000000000000000000000000000000000006000000000000000000088B11
:2B63F100020000000018000000000000000000000000000000000000000000000000000000000000000000000088F4EB
:2B641C00000000000000100000000000000000000000000000000000000000000000004000000000000000000080F392
:2B6447000000000000060000000000000000000000000000000000000000000000008001000000000000000000009E05
:2B647200000000000018000000000000000000000000000000000000000000000000000000000000000000000000FEE9
:2B649D0002000000001C010000000000000000000000000000000000000000000000000104000000000000000088E444
:2B64C800020000000018000000000000000000000000000000000000000000000000000800000000000000000008F48B
:2B64F300040000000018000000000000000000000000000000000000000000000000000000000000000000000010EB67
:2B651E00020000000000000000000000000000000000000000000000000000000000000000000000000000000008ED5B
:2B6549000200000000000000000000000000000000000000000000000000000000000006000000000000000000088B8C
:2B657400020000000010100000000000000000000000000000000000000000000000002000000000000000000008EEC4
:2B659F00000000000016000000000000000000000000000000000000000000000000800500000000000000000000CB6B
:2B65CA00000000000010000000000000000000000000000000000004000000000000008600000000000000000080D8B4
:2B65F500000000000014010000000000000000000000000000002000000000000000000500000000000000000080E0E1
:2B6620000200000000100400000000000000000000000000000080000000000000000006000000000000000000089615
:2B664B00020000000010000000000000000000000000000000000000000000000000008400000000000000000008B0D6
:2B667600040000000010020000000000000000000000000000002000000000000000000002000000000000000090C36E
:2B66A1000200000000280000000000000000000000000000000000000000000000000004000000000000000000888395
:2B66CC00020000000000000000000000000000000000000000000000000000000000002000000000000000000008EF8A
:2B66F700020000000086000000000000000000000000000000000004000000000000800100000000000000000008D48F
:2B672200000000000000000000000000000000000000000000004000000000000000008000000000000000000080EB21
:2B674D0000000000001C020000000000000000000000000000000000000000000000000100000000000000000000AD55
:2B677800000000000018040000000000000000000000000000000000000000000000000004000000000000000000BA1C
:2B67A300000000000038000000000000000000000000000000000000000000000000000800000000000000000008D4AF
:2B67CE00020000000000000000000000000000000000000000000000000000000000000000000000000000000008EDA9
:2B67F900020000000018000000000000000000000000000000000000000000000000000C04000000000000000090E9D2
:2B682400020000000000100000000000000000000000000000000000000000000000000000000000000000000008FD32
:2B684F0002000000001600000000000000000000000000000000000000000000000080290000000000000000000887CE
:2B687A00000000000018000000000000000000000000000000000000000000000000000000000000000000000088F65D
:2B68A500000000000014010000000000000000000000000000000000000000000000008700000000000000000080C8E4
:2B68D000000000000018000000000000000000000000000000000000000000000000000602000000000000000000B8C5
:2B68FB00000000000010020000000000000000000000000000000000000000000000000E0000000000000000000092C0
:2B692600020000000020000000000000000000000000000000000000000000000000000000000000000000000008CF4D
:2B6951000200000000100000000000000000000000000000000000000000000000000006000000000000000000089A61
:2B697C00040000000000100000000000000000000000000000000000000000000000002000000000000000000090E04C
:2B69A70002000000001E0000000000000000000000000000000000000000000000008001000000000000000000088D8F
:2B69D2000200000000000000000000000000000000000000000000000000000000000086000000000000000000088387
:2B69FD0002000000001C010000000000000000000000000000000000000000000000000700000000000000000088C2FF
:2B6A28000000000000000400000000000000000000000000000020000000000000000006000000000000000000808712
:2B6A53000000000000180000000000000000000000000000000000000000000000000006000000000000000000009862
:2B6A7E00000000000018000000000000000000000000000000000000000000000000000000000000000000000000FED7
:2B6AA900000000000000000000000000000000000000000000000000000000000000000000000000000000000080E75B
:2B6AD400020000000000000000000000000000000000000000000000000000000000002000000000000000000008EF7E
:2B6AFF00020000000006040000000000000000000000000000000000000000000000800700000000000000000088F65B
:2B6B2A00020000000000000000000000000000000000000000000000000000000000008000000000000000000008E5D1
:2B6B550002000000001C020000000000000000000000000000000000000000000000000700000000000000000088C1A5
:2B6B8000000000000018080000000000000000000000000000000000000000000000000004000000000000000000B610
:2B6BAB00000000000038000000000000000000000000000000000000000000000000000E00000000000000000080BA3F
:2B6BD600000000000000000000000000000000000000000000000000000000000000000600000000000000000080818D
:2B6C0100000000000018000000000000000000000000000000000000000000000000000000000000000000000000FE52
:2B6C2C000A0000000000000000000000000000000000000000000000000000000000000000000000000000000008E546
:2B6C5700000000000000000000000000000000000000000000000000000000000000000000000000000000000080E7AB
:2B6C8200800008800008800008800008800008800008000000000020000220000220000220000220000220000280E784
:2B6CAD00800008800008800008800008800008800008000000000020000220000220000220000220000220000280E759
:2B6CD800000000002000000000000000000000000000000000000000000000000040000004000000000000000080E1CC
:2B6D0300000000000000040000000000000000000000000000000000000000000000000000000000000000000080E3FE
:2B6D2E00200000000010000000000000200000000000800401400000800008800040000000000000000000000080A6B7
:2B6D5900000000002000000000000000008000000000000000000000000000000000008200000000000000000080C7A6
:2B6D8400200000000008040000000000208000000000408200200000800008800000000004000000000000000080E1C9
:2B6DAF00000000000010000000000000000000000000400001000000000000000000000104000000000000000080F7EC
:2B6DDA00000000000000000000000000000000000000008000000000000000000000000002000000000000000080CFBD
:2B6E0500000000000000000000000000000000000000000000000000000000000000000000000000000000000080E7FB
:2B6E3000000000000000000000000000000000000000000000000000000000000000000000000000000000000080E7D0
:2B6E5B00040000000000000000000000000000000000000000000000000000000000000002000000000000000080C3C3
:2B6E8600140000000000050000000000000000000000000000000000000000000000008001000000000000000080EED9
:2B6EB1000000000000000000000000000000000000000000000000000000000000000000000000000000000000D0B234
:2B6EDC00000000000000000000000000000000000000000000000000000000000000000000000000000000000080E724
:2B6F0700000000000004000000000000000000000000000000000000000000000000000000000000000000000080A734
:2B6F3200000000000000000000000000000000000000000000000000000000000000000000000000000000000080E7CD
:2B6F5D00000000000000000000000000000000000000000000000000000000000000000000000000000000000080E7A2
:2B6F8800000000000000000000000000000000000000000000000000000000000000000000000000000000000080E777
:2B6FB3000000000000000000000000000000000000000000000000000000000000000000000000000000000000A0C54E
:2B6FDE00000000000080100000000000000000000000000000000000000000000000000000000000000000000000F701
:2B70090000008002408810108800208800000080002010000000000000000020400000020080A0040000000000008408
:2B703400000000820008022048822001020000002008020000000000000000088000008000008200000000000000994B
:2B705F00000000000000000000000000000000000000000000000000000000000000000000000000000000000080E79F
:2B708A00000000000000000000000000000000000000000000000000000000000000000000000000000000000080E774
:2B70B500A0288AE3288EA3388EE3388AA3280AA1388E03000000001084A2288EE22804E12884E3108A42100441808ECF
:2B70E000C075DD657197C55D966559BCC575DDC15D9605000000001806D7751777718761718765195C7718866180BF2C
:02710B00FFFF84
:00000001FF
